:100000000C9465020C94AC020C94AC020C94AC02FF
:100010000C94AC020C94AC020C94AC020C94AC02A8
:100020000C94AC020C94AC020C94C50B0C94970C81
:100030000C94AC020C94AC020C94AC020C94AC0288
:100040000C94AC020C940B210C94AC020C94AC02FA
:100050000C94AC020C949D1A0C94AC020C94AC025F
:100060000C94AC020C94AC020C94AC020C94AC0258
:100070000C94AC020C94AC020C94AC020C94AC0248
:100080000C94AC020C94AC020C94AC020C94AC0238
:100090000C94AC020C94AC020C94AC020C94AC0228
:1000A0000C94AC020C94AC020C94AC02040D260D22
:1000B000190E260D190E6B0D8E0D190EE30DF60D92
:1000C000E010E0100F110F1152118C1199139913B8
:1000D000A51199139A129A126D13991399138413F7
:1000E0000000F0A123024C003900E100648100000F
:1000F0001E00140004001D0031714D001F001A0085
:1001000016001B002E002A00200008000700060031
:1001100038002C00210015000900190030004A00A9
:10012000220017000A00050000006574AE000154AB
:100130000000007F0000E300AB00025400000077E5
:100140000000E20023001C000B00110000002971D8
:10015000240018000D00100050004B0025000C007A
:100160000E00360051002800260012000F00370054
:1001700052002B0027001300330038714F004E004F
:100180002D002F003482E500C100000001000100B5
:1001900001000100010000003A001E0231002202AD
:1001A000010001003B001414210235000100010090
:1001B0003C00241425022514010001003D002714F1
:1001C00026022614010001003E0064142E023014A1
:1001D000000001000100010000000100000001001A
:1001E0000100010000000100000001003F0052007A
:1001F00051002302000001004000240021001E00E5
:10020000010001004100250022001F00370001000D
:100210004200260023002000270001004300300296
:1002200030002D14270201004400450001000100A8
:1002300001000000010001000100010001000000B8
:100240003A000100F700FB00010001003B00F40050
:10025000F200FA00FD00F5003C00F000F100F900AA
:10026000FE00F4003D00F500F300FC00FF0001007B
:100270003E000100F800F60000000100010001004E
:100280000000010000000100010001000000010069
:10029000000001003F0001000100B4000000010067
:1002A0004000AA00AC00B600010001004100A80017
:1002B000AD00B5000100B7004200A900AE00B900D2
:1002C0000100B60043000100AB00B70001000100CF
:1002D0004400450001000100010000001603450034
:1002E000720067006F0044006F0078002000450036
:1002F0005A00000016034500720067006F004400BA
:100300006F007800200045005A0000000403090433
:1003100009026D00040100A0FA09040000010301B4
:100320000100092111010001223F00070581030896
:10033000000A090401000103010200092111010062
:1003400001224D000705820308000A09040200018A
:100350000300000009211101000122360007058376
:100360000308000A09040300010300000009211129
:100370000100012239000705840310000112011059
:100380000100000008EDFE07130100010200010555
:10039000010906A101050719E029E71500250195C6
:1003A0000875018102050819012905950575019156
:1003B000029501750391010507190029771500259C
:1003C00001957875018102C005010980A1018502AE
:1003D00016010026B7001A01002AB7007510950112
:1003E0008100C0050C0901A1018503160100269CAE
:1003F000021A01002A9C02751095018100C00501B6
:100400000902A1010901A100050919012905150029
:10041000250195057501810295017503810105018D
:10042000093009311581257F950275088106093843
:100430001581257F950175088106050C0A3802157E
:1004400081257F950175088106C0C005010906A1B7
:1004500001050719E029E7150025019508750181B7
:100460000295017508810105081901290595057591
:100470000191029501750391010507190029FF15E6
:100480000025FF950675088100C0000000000000EF
:100490000000000000010204060A0F17202C3A4A4F
:1004A0005D71879DB3C7DAE9F5FCFFFCF5E9DAC7B2
:1004B000B39D87715D4A3A2C20170F0A060402018A
:1004C0000000000000000000000011241FBECFEF5C
:1004D000DAE0DEBFCDBF04B603FE27C08091ED0198
:1004E0009091EE01A091EF01B091F0018730904B17
:1004F000A740B04BD1F41092ED011092EE01109292
:10050000EF011092F00114BE84B7877F84BF0FB64D
:10051000F894A895809160008861809360001092A3
:1005200060000FBEE0E0FFE3099511E0A0E0B1E05C
:10053000E8EBF5E402C005900D92A433B107D9F7BA
:1005400021E0A4E3B1E001C01D92AD3EB207E1F7A6
:100550000E940C090C94DA220C94000061110BC06B
:10056000FC018281882321F085EE0E947A0F03C06E
:1005700085EE0E94421080E090E008950895609119
:10058000B1017091B2018091B3019091B4010E94C8
:10059000CA1956985E9825982D9826982E982798CF
:1005A0002F98813029F0823031F4269A2E9A0895BE
:1005B000259A2D9A089556985E9808950C94BF0236
:1005C00056985E9825982D9826982E9827982F98BB
:1005D0008FEF90E0909389008093880090938B0038
:1005E00080938A0090938D0080938C00259A2D9A99
:1005F0002FEF80E792E0215080409040E1F700C06B
:100600000000269A2E9A2FEF80E792E0215080403A
:100610009040E1F700C00000279A2F9A2FEF80E763
:1006200092E0215080409040E1F700C00000259802
:100630002D982FEF80E792E0215080409040E1F725
:1006400000C0000026982E982FEF80E792E02150FE
:1006500080409040E1F700C0000027982F985698FE
:100660005E9825982D9826982E9827982F9808956B
:1006700089EA8093800089E08093810024982C98F7
:100680003F988AB18F748AB96E98479A8BB1806B04
:100690008BB9769A0E94E0020C94BE0280E28093AD
:1006A00000018091340181110EC00E949D0381E000
:1006B000809334012FEF83ED90E3215080409040F0
:1006C000E1F700C0000080E40E94A30380930001D2
:1006D00081112EC00E94CD0380930001811128C09A
:1006E0000E94CD0380930001811122C08FE30E94FC
:1006F000CD038093000181111BC00E94C50380E4DB
:100700000E94A30380930001811112C08CE00E941B
:10071000CD038093000181110BC00E94CD03809313
:100720000001811105C08FE30E94CD038093000179
:100730000E94C5038091000108951092B9008AE0DB
:100740008093B800089594EA9093BC009091BC0007
:1007500097FFFCCF9091B900987F983021F09031AD
:1007600011F081E008958093BB0084E88093BC0081
:100770008091BC0087FFFCCF8091B900887F8831D1
:1007800011F0803471F780E0089584E98093BC0013
:100790008091BC0084FDFCCF08958093BB0084E869
:1007A0008093BC008091BC0087FFFCCF9091B90082
:1007B000987F81E0983209F480E0089584E880937E
:1007C000BC008091BC0087FFFCCF8091BB000895E6
:1007D00080910001811115C080E40E94A3038093E1
:1007E000000181110CC082E10E94CD0380930001C1
:1007F000811105C08FEF0E94CD03809300010E94FC
:10080000C50384B1807F84B985B1807F85B98AB101
:10081000837F8AB98BB1837F8BB93E9846980895C0
:100820000E944E03809300010E94E80380B38C7005
:1008300080BB81B3836F81BBE4E4F1E0A6E3B1E068
:1008400011921D9281E0E235F807D1F70C9438033C
:100850009F92AF92BF92CF92DF92EF92FF920F934F
:100860001F93CF93DF9380910001882379F08091CB
:1008700035018F5F80933501811108C00E944E03BE
:1008800080930001811102C00E94E00286E3E82EFD
:1008900081E0F82E8701C0E0D0E0BB24B39492E061
:1008A000A92ECC24C394D12CC730D10500F580915A
:1008B0000001811164C080E40E94A30380930001C1
:1008C000811112C082E10E94CD0380930001811149
:1008D0000BC0C6010C2E01C0880F0A94EAF7809560
:1008E0000E94CD03809300010E94C50348C0CA3016
:1008F000A1F028F4C83059F0C93061F005C0CC30FF
:1009000089F070F0CD3089F0209A289810C0219A93
:1009100029980DC0229A2A980AC0239A2B9807C0BA
:10092000529A01C0539A5B9802C03E9A4698E0EAF8
:10093000EA95F1F78FB181708B25799902C032E089
:1009400001C030E0832B7C9902C034E001C030E06C
:10095000832B7D9902C028E001C020E0822B7E9984
:1009600002C090E101C090E0892B9FB19095991F42
:100970009927991F9295990F907E892B0FC080918E
:10098000000181114AC080E40E94A303809300010A
:10099000882381F1912C0E94C503892DD8019C9157
:1009A000981719F08C93A09201010E94E8032196F8
:1009B0000F5F1F4FCE30D10509F076CF8091010136
:1009C000882369F1815080930101882339F0EFE990
:1009D000FFE03197F1F700C0000021C0E4E4F1E04E
:1009E000D7018D917D018193B4E4EB16B1E0FB0654
:1009F000B9F715C083E10E94CD03809300018111F6
:100A0000C9CF81E40E94A303809300018111C2CF6A
:100A10000E94DE03982E9094BECF80E0BFCF0E944C
:100A2000DE0281E0DF91CF911F910F91FF90EF9057
:100A3000DF90CF90BF90AF909F900895E82FF0E0A7
:100A4000EC5BFE4F8081089508958B3B910580F407
:100A5000883A910548F5853A9105D8F48430910596
:100A600008F0B2C0019709F06EC081E090E00895EF
:100A7000803E910508F467C0883E910508F4A4C043
:100A80009C01205F31092031310508F05CC0906580
:100A90000895853A910509F459C0863A910509F0FF
:100AA00058C082E890E40895883A910509F454C04A
:100AB000893A910509F453C08A3A910509F452C064
:100AC0008B3A910509F451C08C3A910509F450C054
:100AD0008D3A910509F44FC0803B910509F44EC051
:100AE0008E3A910509F44DC08F3A910509F44CC036
:100AF000813B910509F44BC0823B910509F44AC042
:100B0000833B910509F449C0843B910509F448C031
:100B1000853B910509F447C0863B910509F446C021
:100B2000873B910509F445C0883B910509F444C011
:100B3000893B910509F443C08A3B910509F442C001
:100B400080E094E4089580E090E0089581E890E4E6
:100B5000089583E890E4089582EE94E4089589EE80
:100B600094E408958AEE94E4089585EB94E408955E
:100B700086EB94E4089587EB94E408958CEC94E478
:100B800008958DEC94E4089583E895E408958AE847
:100B900095E4089582E995E4089584E995E408953B
:100BA00081E296E4089583E296E4089584E296E46F
:100BB000089585E296E4089586E296E4089587E232
:100BC00096E408958AE296E40895089524E5829FC4
:100BD000C0011124FC0126E0729FE00DF11D1124DB
:100BE000E60FF11DEE0FFF1FEC51FF4F8591949121
:100BF0000895880F991FFC01E05AF0408591949167
:100C00000895880F991FFC01E052FF4F8591949140
:100C1000089524E5829FC0011124FC0146E0749FE1
:100C2000E00DF11D1124E60FF11DEE0FFF1FEC5139
:100C3000FF4F859194919C013A9521154FE134071E
:100C400008F425C13F512115304120F49F700E94C6
:100C5000010608959C0130532115304118F499275D
:100C6000906C0895811520E5920769F40E94BB13EA
:100C70004FEF84E39CE0415080409040E1F700C09A
:100C800000000C94C21A813020E5920731F4809163
:100C9000CC0181608093CC0108959C0130552115D1
:100CA000304108F05CC0292F33272F7033272130C3
:100CB0003105E9F4AC0164E0440F551F6A95E1F792
:100CC00044275370BC016370772702C0220F331F83
:100CD0006A95E2F73C68242B352B73E0880F991F47
:100CE0007A95E1F780769927822B932B089522300D
:100CF000310529F4982F8827816F906A0895233051
:100D00003105A1F4AC0133E0440F551F3A95E1F7EA
:100D1000407E57708370992721E030E002C0220F97
:100D2000331F8A95E2F7C9019C6816C0243031054B
:100D300031F5AC0123E0440F551F2A95E1F7407EC1
:100D400057708370992721E030E002C0220F331FD3
:100D50008A95E2F7C9019A68842B952B08959C0126
:100D600030572115304118F49F70906208959C010E
:100D700030582115304118F49F70906A0895803ED4
:100D80009105E0F4803C910558F58133910509F413
:100D90006FC048F48932910509F463C08A32910525
:100DA00009F46DC072C089339105E9F0823891056C
:100DB000D1F08533910509F44DC067C0833E91059C
:100DC00081F138F4803E9105B9F0823E9105D9F069
:100DD0005CC0863E910561F1873E9105A1F155C049
:100DE0000E94F90508952091DE0120FD02C021FF37
:100DF0004CC080EE90E049C08091DE0180FFF9CFC9
:100E000089E390E042C08091DE0182FF0EC08091B4
:100E1000DE0184FF03C080E090E037C083EE90E005
:100E200034C08091DE0182FFF2CF82EE90E02DC0CF
:100E30008091DE0183FF0BC08091DE0184FDEBCF4A
:100E400087EE90E022C08091DE0183FFF5CF86EE31
:100E500090E01BC08091DE0185FF07C089E290E031
:100E600014C08091DE0185FFF9CF85E390E00DC0CD
:100E70008091DE0186FF07C08AE290E006C0809183
:100E8000DE0186FFF9CF81E390E00E9425050895F9
:100E90000895809162010895CF93DF9300D01F924F
:100EA000CDB7DEB79C018091E401843019F593E061
:100EB00099833B832A839093E9008FEF9091E80018
:100EC000815095FD06C095ED9A95F1F700008111CE
:100ED000F5CF8091E80085FF0DC040E050E063E071
:100EE00070E0CE0101960E94B9098091E8008E77EA
:100EF0008093E8000F900F900F90DF91CF910895AD
:100F0000CF93DF9300D01F92CDB7DEB72091E401DD
:100F1000243021F522E029839B838A8383E0809318
:100F2000E9008FEF9091E800815095FD06C095EDA6
:100F30009A95F1F700008111F5CF8091E80085FFC7
:100F40000DC040E050E063E070E0CE0101960E94E9
:100F5000B9098091E8008E778093E8000F900F9098
:100F60000F90DF91CF9108959C018091E40184302E
:100F7000F9F482E08093E9009FEF8091E8009150BE
:100F800085FD06C085ED8A95F1F700009111F5CF3A
:100F90008091E80085FF0CC040E050E065E070E023
:100FA000C9010E94B9098091E8008E778093E8001A
:100FB0000895CF93DF93EC018091E401843009F030
:100FC00046C090910C019923D9F090910D0199237D
:100FD000B9F08093E9008FEF9091E800815095FD82
:100FE00006C095E19A95F1F700008111F5CF809147
:100FF000E80085FF2CC040E050E060E170E017C0E1
:1010000081E08093E9008FEF9091E800815095FD99
:1010100006C095ED9A95F1F700008111F5CF80910A
:10102000E80085FF14C040E050E068E070E0CE01C9
:101030000E94B9098091E8008E778093E80080E1F2
:10104000FE01A2E5B1E001900D928A95E1F7DF91F2
:10105000CF9108958091E301811109C00E944A0B4C
:101060000E94A70B8091E20084608093E2000895C3
:101070001092E301089508950C94F8200E94581AE4
:101080000E94FE200E94520E0C94480742E061EC40
:1010900081E00E94C30A42E061EC82E00E94C30A40
:1010A00042E061EC83E00E94C30A42E161EC84E02B
:1010B0000C94C30A8091E601833009F455C030F4E2
:1010C000813071F0823009F48EC008958A3009F4BD
:1010D0007AC08B3009F460C0893009F09CC020C010
:1010E0008091E501813A09F096C08091E800877F00
:1010F0008093E8008091E9019091EA01892B21F425
:1011000060E182E591E003C060E080E090E070E0A3
:101110000E94040A8091E8008B778093E80008958C
:101120008091E501813209F076C08091E9019091CA
:10113000EA01009719F0039709F06DC08091E8006B
:10114000877F8093E8008091E80082FD05C0809150
:10115000E4018111F8CF5FC08091F10080936201BA
:101160008091E8008B7753C08091E501813A09F0C6
:1011700052C08091E9019091EA01892B09F04BC09E
:101180008091E800877F8093E8008091E80080FFED
:10119000FCCF80910C0136C08091E5018132D9F5F8
:1011A0008091E9019091EA01892BA9F58091E800ED
:1011B000877F8093E8000E94F80A8091E70180937E
:1011C0000C010C94BB138091E501813221F58091D3
:1011D000E800877F8093E8000E94F80A8091E80188
:1011E0008093630108958091E501813AA1F4809193
:1011F000E800877F8093E8008091E80080FFFCCFC3
:10120000809163018093F1008091E8008E77809354
:10121000E8000C94F80A089584B7877F84BF0FB65E
:10122000F894A89580916000886180936000109286
:1012300060000FBE90E080E80FB6F89480936100E4
:10124000909361000FBE0E94A10E0E944A0B0E9463
:10125000A70B8091E20084608093E20078940E9462
:10126000320E0E94A30E82E091E00E944D0E0E9479
:10127000E6208091E401853069F40E941A1A809179
:10128000E2018823B1F30E94441A882391F30E945B
:10129000A309EFCF0E94A90EECCF292F33272330CB
:1012A0003105C9F060F42130310581F0223031057B
:1012B00009F041C08DE690E020E133E040C02132EA
:1012C0003105E1F02232310531F135C082E190E0A3
:1012D0002DE733E034C099278130910549F028F09B
:1012E000029749F5ECEDF2E005C0ECE0F3E002C056
:1012F000E4EFF2E0849190E09F0121C06430D8F4E3
:10130000E62FF0E0EE0FFF1FEE5DFE4F20813181F2
:1013100089E090E014C0643070F470E0FB01EE0FDF
:10132000FF1FE65EFE4F20813181FB01EA5EFE4F2A
:10133000808190E004C080E090E020E030E0FA019D
:1013400031832083089580E189BD82E189BD09B49C
:1013500000FEFDCF8091D8008F7D8093D8008091D2
:10136000E00082608093E0008091E00081FDFCCF8E
:101370000895CF92DF92EF92FF920F931F93CF9336
:10138000DF93EC018B016A010E94170B811133C0BE
:10139000C114D10439F0F60180819181081B190B29
:1013A000C80FD91FE12CF12C0115110519F18091FD
:1013B000E80085FD16C08091E8008E778093E800F4
:1013C000C114D10449F0F60180819181E80EF91E23
:1013D000F182E08285E00FC00E94170B882321F381
:1013E0000AC089918093F10001501109FFEFEF1AB3
:1013F000FF0ADACF80E0DF91CF911F910F91FF902C
:10140000EF90DF90CF9008952091EB013091EC01A7
:101410002617370748F06115710539F42091E80067
:101420002E772093E80001C0B901FC0120E061158E
:10143000710579F18091E4018823F1F18530F1F1B2
:101440008091E80083FD3CC08091E80082FD2EC0C1
:101450008091E80080FFEBCF2091F3008091F200B3
:1014600090E0922B6115710551F08830910538F4A8
:1014700021912093F100615071090196F3CF21E091
:10148000089709F020E08091E8008E778093E800CB
:10149000CECF2111CFCF0AC08091E401882361F023
:1014A000853061F08091E80083FD0AC08091E800FA
:1014B00082FFF2CF80E0089582E0089583E00895EE
:1014C00081E008952091EB013091EC012617370758
:1014D00048F06115710539F42091E8002E772093CA
:1014E000E80001C0B901FC0120E06115710591F12E
:1014F0008091E401882309F440C0853009F43FC09D
:101500008091E80083FD3DC08091E80082FD2FC0FE
:101510008091E80080FFE9CF2091F3008091F200F4
:1015200090E0922B6115710559F08830910540F4D7
:1015300024912093F1003196615071090196F2CF08
:1015400021E0089709F020E08091E8008E778093F1
:10155000E800CBCF2111CCCF0AC08091E4018823D1
:1015600061F0853061F08091E80083FD0AC08091D0
:10157000E80082FFF2CF80E0089582E0089583E0E2
:10158000089581E00895982F973068F59093E900C9
:10159000981739F07091EC002091ED005091F00017
:1015A00003C0242F762F50E021FD02C09F5FECCFB7
:1015B0003091EB003E7F3093EB003091ED003D7FAA
:1015C0003093ED003091EB0031603093EB0070937D
:1015D000EC002093ED005093F0002091EE0027FDE9
:1015E000E5CF80E008958F708093E90081E0089551
:1015F0008091E50187FF11C08091E80082FD05C060
:101600008091E4018111F8CF11C08091E8008B77BF
:101610000BC08091E401882349F08091E80080FFAD
:10162000F8CF8091E8008E778093E80008952091AC
:10163000E4003091E50095E64091EC00842F817044
:1016400040FF23C08091E80080FD1DC08091E4012F
:10165000882399F0853099F08091EB0085FD11C0C9
:101660004091E4005091E5002417350729F391508B
:1016700011F09A01E1CF84E0089582E0089583E0BB
:10168000089581E0089580E008954091E80042FFC8
:10169000DDCF08950E94B80B0E94C00BE0EEF0E091
:1016A000808181608083E8EDF0E080818F778083A6
:1016B00019BCA7EDB0E08C918E7F8C9380818F7EDA
:1016C00080831092E30108950F931F93CF93DF93CC
:1016D0000E94B80B0E94C00BC8EDD0E088818F77C4
:1016E000888388818068888388818F7D888319BCFE
:1016F0001092E4011092E0011092E2011092E101D7
:1017000000EE10E0F80180818B7F8083888181600A
:10171000888342E060E080E00E94C30AE1EEF0E0EE
:1017200080818E7F8083E2EEF0E080818160808323
:10173000808188608083F80180818E7F80838881AA
:1017400080618883DF91CF911F910F910895E8ED1B
:10175000F0E080818F7E8083E7EDF0E08081816022
:10176000808384E082BF81E08093E3010C94640B6A
:10177000E8EDF0E080818E7F80831092E200089592
:101780001092DA001092E10008951F920F920FB6A6
:101790000F9211242F933F934F935F936F937F93F7
:1017A0008F939F93AF93BF93EF93FF938091E1004B
:1017B00082FF0BC08091E20082FF07C08091E100B0
:1017C0008B7F8093E1000E94310E8091DA0080FFD0
:1017D0001FC08091D80080FF1BC08091DA008E7FEF
:1017E0008093DA008091D90080FF0DC080E189BD2F
:1017F00082E189BD09B400FEFDCF81E08093E40160
:101800000E942A0805C019BC1092E4010E94380801
:101810008091E10080FF19C08091E20080FF15C037
:101820008091E2008E7F8093E2008091E2008061EF
:101830008093E2008091D80080628093D80019BC28
:1018400085E08093E4010E943C088091E10084FFE0
:1018500030C08091E20084FF2CC080E189BD82E12C
:1018600089BD09B400FEFDCF8091D8008F7D8093A3
:10187000D8008091E1008F7E8093E1008091E200AA
:101880008F7E8093E2008091E20081608093E2008D
:101890008091E001882311F084E007C08091E3008B
:1018A00087FD02C081E001C083E08093E4010E94D3
:1018B0003E088091E10083FF29C08091E20083FF10
:1018C00025C08091E100877F8093E10082E08093D2
:1018D000E4011092E0018091E1008E7F8093E100AD
:1018E0008091E2008E7F8093E2008091E20080612F
:1018F0008093E20042E060E080E00E94C30A8091B1
:10190000F00088608093F0000E943B08FF91EF9107
:10191000BF91AF919F918F917F916F915F914F9107
:101920003F912F910F900FBE0F901F9018951F920F
:101930000F920FB60F9211242F933F934F935F9303
:101940006F937F938F939F93AF93BF93CF93DF93C7
:10195000EF93FF93C091E900CF708091EC00D82FF6
:10196000D17080FDD0E81092E9008091F000877F6F
:101970008093F00078940E94DB0C1092E900809133
:10198000F00088608093F000CD2BCF70C093E90009
:10199000FF91EF91DF91CF91BF91AF919F918F9187
:1019A0007F916F915F914F913F912F910F900FBE5B
:1019B0000F901F9018951F93CF93DF93CDB7DEB78D
:1019C000AA970FB6F894DEBF0FBECDBFE5EEF1E0EB
:1019D0008091F100819321E0ED3EF207C9F70E946A
:1019E0005A088091E80083FF24C18091E50190911D
:1019F000E601492F50E04A30510508F01AC1FA01BA
:101A0000EA5AFF4F0C948F22803881F0823809F017
:101A100010C18091E9018F708093E9008091EB0003
:101A200085FB882780F91092E90006C08091E101CA
:101A30009091E201911182609091E800977F9093DC
:101A4000E8008093F1001092F100C8C0282F2D7F8C
:101A500009F0EFC0882319F0823061F0EAC080916C
:101A6000E701813009F0E5C0933009F080E0809310
:101A7000E2012BC08091E701811127C08091E9012B
:101A80008F7009F4D6C08093E9002091EB0020FF0D
:101A90001CC0933021F48091EB00806214C09091BF
:101AA000EB0090619093EB0021E030E0A90102C0CF
:101AB000440F551F8A95E2F74093EA001092EA001E
:101AC0008091EB0088608093EB001092E900809198
:101AD000E800877F86C08111ACC01091E7011F77B5
:101AE0008091E3008078812B8093E3008091E8006F
:101AF000877F8093E8000E94F80A8091E80080FFC9
:101B0000FCCF8091E30080688093E300111102C054
:101B100082E001C083E08093E4018BC08058823072
:101B200008F087C08091E7019091E8018C3D53E077
:101B3000950779F583E08A838AE289834FB7F89421
:101B4000DE01139620E03EE051E2E32FF0E05093F7
:101B50005700E49120FF03C0E295EF703F5FEF7004
:101B60008E2F90E0EA3010F0C79601C0C0968D939A
:101B70009D932F5F243149F74FBF8091E800877F05
:101B80008093E8006AE270E0CE0101960E94040AA8
:101B900014C0AE014F5F5F4F6091E9010E944D0993
:101BA000BC01892B09F445C09091E800977F909380
:101BB000E80089819A810E94620A8091E8008B770F
:101BC0008093E80036C08038A1F58091E800877FD7
:101BD0008093E8008091E0018093F1008091E8001B
:101BE0008E778093E8000E94F80A23C0811121C0FB
:101BF0008091E7019091E80199270297D4F48091B0
:101C0000E800877F8093E8008091E7018093E001FE
:101C10000E94F80A8091E001811106C08091E300E2
:101C200087FD02C081E001C084E08093E4010E944E
:101C300046088091E80083FF0AC08091E800877F12
:101C40008093E8008091EB0080628093EB00AA967D
:101C50000FB6F894DEBF0FBECDBFDF91CF911F91BD
:101C600008950895CF938091E4018823A1F0C09155
:101C7000E900CF709091EC00892F817090FD80E891
:101C8000C82B1092E9008091E80083FD0E94DB0CD4
:101C9000CF70C093E900CF9108959093690180932C
:101CA00068010895E0916801F0916901309721F091
:101CB0000190F081E02D099480E00895E0916801A1
:101CC000F0916901309721F00280F381E02D0994B1
:101CD0000895E0916801F0916901309721F0048046
:101CE000F581E02D099408952091660130916701F6
:101CF0002817390771F09093670180936601E0918E
:101D00006801F0916901309721F00680F781E02D9C
:101D100009940895209164013091650128173907CD
:101D200071F09093650180936401E0916801F091F6
:101D30006901309721F00084F185E02D0994089520
:101D400008950C94A00E0E945E1A0E9410040C9438
:101D5000241BCF92DF92EF92FF920F931F93CF93AA
:101D6000DF93CDB7DEB72B970FB6F894DEBF0FBE6B
:101D7000CDBF0E9428048BE6C82E81E0D82E00E05B
:101D800010E0E02E802F0E941E05F60141916F01A8
:101D9000F82EF426B1F40F5F1F4F0E30110589F7AE
:101DA0008FEF89838A831B820E94671A8160782F54
:101DB0009D838C8349815A816B818D810E944C0F58
:101DC00040C09091CC0191FF04C08B870E942405F4
:101DD0008B8520E030E04F2D50E0922FBA01022E8B
:101DE00002C0759567950A94E2F760FF24C02E83C0
:101DF000EF8221E030E0690102C0CC0CDD1C9A9535
:101E0000E2F790E08C219D21892B09F420E02887BE
:101E10000E94671A8160782F9A8789874E815F8137
:101E200068858A850E944C0FF801E559FE4F808134
:101E3000C826C08206C02F5F3F4F2630310569F6A5
:101E4000AACF0E940B1E0E94520E90916A01891720
:101E5000A1F00E94520E80936A012B960FB6F8945F
:101E6000DEBF0FBECDBFDF91CF911F910F91FF90CD
:101E7000EF90DF90CF900C9448072B960FB6F89414
:101E8000DEBF0FBECDBFDF91CF911F910F91FF90AD
:101E9000EF90DF90CF900895CF93DF93CDB7DEB76B
:101EA0002B970FB6F894DEBF0FBECDBF4F83588778
:101EB00069877A878B87DE01119686E0FD01119292
:101EC0008A95E9F785E0FE01379601900D928A9593
:101ED000E1F749815A816B817C818D819E810E94CD
:101EE0004F162B960FB6F894DEBF0FBECDBFDF9115
:101EF000CF910895CF93C82F882309F4C1C08238A9
:101F000059F40E94520E81FDBBC089E30E94EC1877
:101F10000E94A41989E30CC0833879F40E94520E00
:101F200080FDAEC083E50E94EC180E94A41983E5F1
:101F30000E942B19CF910C94A419843859F40E9453
:101F4000520E82FD9DC087E40E94EC180E94A419E5
:101F500087E4EECF8CEF8C0F813A48F48C2F0E94EF
:101F60004B2081118DC08C2F0E94EC18E3CF80E2B2
:101F70008C0F883048F4C77081E001C0880FCA9583
:101F8000EAF70E946D19D6CF8BE58C0F833078F479
:101F9000C53A29F0C63A31F083E890E005C081E8FF
:101FA00090E002C082E890E0CF910C94740E88E536
:101FB0008C0F833108F064C0C83A39F1C93A41F155
:101FC000CA3A49F1CB3A51F1CC3A59F1CD3A61F1E3
:101FD000C03B69F1CE3A71F1CF3A79F1C13B81F161
:101FE000C23B89F1C33B91F1C43B99F1C53BA1F1DF
:101FF000C63BA9F1C73BB1F1C83BB9F1C93BC1F13F
:10200000CA3BC9F180E090E038C082EE90E035C074
:1020100089EE90E032C08AEE90E02FC085EB90E030
:102020002CC086EB90E029C087EB90E026C08CECBA
:1020300090E023C08DEC90E020C083E891E01DC0CB
:102040008AE891E01AC082E991E017C084E991E042
:1020500014C081E292E011C083E292E00EC084E2FB
:1020600092E00BC085E292E008C086E292E005C0F3
:1020700087E292E002C08AE292E0CF910C948A0E4D
:10208000CF910895882309F44BC0823859F40E94F7
:10209000520E81FF45C089E30E94EC180E94A419EA
:1020A00089E30CC0833871F40E94520E80FF38C05F
:1020B00083E50E94EC180E94A41983E50E942B1965
:1020C0000C94A419843859F40E94520E82FF28C03F
:1020D00087E40E94EC180E94A41987E4EFCF9CEFDC
:1020E000980F913A58F390E2980F983050F4877017
:1020F00091E001C0990F8A95EAF7892F0E94731920
:10210000DFCF9BE5980F933020F480E090E00C94B3
:10211000740E885A833120F480E090E00C948A0E8B
:102120000895882321F00E946D190C94A419089534
:10213000882321F00E9473190C94A4190895BF926A
:10214000CF92DF92EF92FF920F931F93CF93DF9383
:1021500000D000D000D0CDB7DEB77C0185E0F7011C
:10216000DE01119601900D928A95E1F7F7018381C6
:102170009481892B09F4DDC2908181818F3F19F40C
:102180009F3F09F4D6C2F7010281258122952F7065
:1021900099838A8389819A812E830E94AB18182F94
:1021A000B92E0E94AA180E947117EB2DE295EF70CC
:1021B0004E2F50E0FA01E05AFF4F2E810C948F22EF
:1021C0008B2D807F9B2D9F70F92E882319F0F29420
:1021D00080EFF822002349F0FF2009F457C28F2D29
:1021E0000E947D190E94A41951C2812F0E944210A1
:1021F000FF2009F49EC28F2D0E94831926960FB6E8
:10220000F894DEBF0FBECDBFDF91CF911F910F912C
:10221000FF90EF90DF90CF90BF900C94A4193B2DCE
:10222000307F8B2D8F70303211F08295807F11239B
:1022300019F0113021F12CC00023B9F0222309F448
:1022400090C1213009F08DC126960FB6F894DEBFFB
:102250000FBECDBFDF91CF911F910F91FF90EF90F7
:10226000DF90CF90BF900C948D19222319F021306C
:1022700009F45FC28E830E9490198E8186C100236B
:1022800021F0223008F055C26CC1211152C27DC12B
:10229000002321F0222309F464C1F8C1222309F4A8
:1022A00074C109C28B2D86958695837019F0813093
:1022B000D1F03FC2002321F0812F9B2D937002C0EB
:1022C00080E090E026960FB6F894DEBF0FBECDBF3B
:1022D000DF91CF911F910F91FF90EF90DF90CF9002
:1022E000BF900C94740E002321F0812F9B2D9370CE
:1022F00002C080E090E026960FB6F894DEBF0FBED5
:10230000CDBFDF91CF911F910F91FF90EF90DF90A4
:10231000CF90BF900C948A0E812F002319F00E9459
:10232000131D02C00E947B1D26960FB6F894DEBFD7
:102330000FBECDBFDF91CF911F910F91FF90EF9016
:10234000DF90CF90BF900C94001E8B2D837009F00E
:1023500075C00111EEC1812F829586958770880F17
:10236000880F912F9F70C92ED12CE12CF12C082EB3
:1023700004C0CC0CDD1CEE1CFF1C0A94D2F714FF29
:1023800012C00FE010E020E030E004C0000F111F89
:10239000221F331F8A95D2F7C901B8016095709545
:1023A0008095909503C060E070E0CB014B2D469581
:1023B000469543704230C1F060F56C297D298E2925
:1023C0009F29413051F126960FB6F894DEBF0FBE1B
:1023D000CDBFDF91CF911F910F91FF90EF90DF90D4
:1023E000CF90BF900C9498176C297D298E299F2936
:1023F00026960FB6F894DEBF0FBECDBFDF91CF910A
:102400001F910F91FF90EF90DF90CF90BF900C94B1
:10241000B4170E949817C701B60126960FB6F89414
:10242000DEBF0FBECDBFDF91CF911F910F91FF9007
:10243000EF90DF90CF90BF900C947C17002319F0A1
:102440008B2D817001C08695882309F472C1812F7C
:10245000829586958770880F880F912F9F70C92E5F
:10246000D12CE12CF12C082E04C0CC0CDD1CEE1C70
:10247000FF1C0A94D2F714FF12C00FE010E020E016
:1024800030E004C0000F111F221F331F8A95D2F7BE
:10249000C901B801609570958095909503C060E082
:1024A00070E0CB014B2D4695469543704230C1F00C
:1024B00060F56C297D298E299F29413051F126969E
:1024C0000FB6F894DEBF0FBECDBFDF91CF911F9145
:1024D0000F91FF90EF90DF90CF90BF900C94721807
:1024E0006C297D298E299F2926960FB6F894DEBF88
:1024F0000FBECDBFDF91CF911F910F91FF90EF9055
:10250000DF90CF90BF900C948E180E947218C70174
:10251000B60126960FB6F894DEBF0FBECDBFDF9191
:10252000CF911F910F91FF90EF90DF90CF90BF90D0
:102530000C945618103FD1F118F4103E50F4A1C07D
:10254000123F09F463C008F44CC0133F09F473C090
:1025500098C01F708B2D8F710023A1F00E94EF1780
:10256000812F26960FB6F894DEBF0FBECDBFDF9148
:10257000CF911F910F91FF90EF90DF90CF90BF9080
:102580000C9491100E941018812F26960FB6F89483
:10259000DEBF0FBECDBFDF91CF911F910F91FF9096
:1025A000EF90DF90CF90BF900C9498100023A9F08B
:1025B0002111BFC08B2D8F7126960FB6F894DEBF08
:1025C0000FBECDBFDF91CF911F910F91FF90EF9084
:1025D000DF90CF90BF900C943518223008F0A9C03E
:1025E000E9CF0023A9F08B2D8F7126960FB6F894B2
:1025F000DEBF0FBECDBFDF91CF911F910F91FF9036
:10260000EF90DF90CF90BF900C94EF17002359F319
:102610008B2D8F7126960FB6F894DEBF0FBECDBFFF
:10262000DF91CF911F910F91FF90EF90DF90CF90AE
:10263000BF900C941018002399F08B2D8F71269663
:102640000FB6F894DEBF0FBECDBFDF91CF911F91C3
:102650000F91FF90EF90DF90CF90BF900C94DA171E
:1026600026960FB6F894DEBF0FBECDBFDF91CF9197
:102670001F910F91FF90EF90DF90CF90BF900C943F
:10268000D0170023A9F0222309F4ADCF812F26967D
:102690000FB6F894DEBF0FBECDBFDF91CF911F9173
:1026A0000F91FF90EF90DF90CF90BF900C947A0F36
:1026B000222309F4ADCF812F26960FB6F894DEBF02
:1026C0000FBECDBFDF91CF911F910F91FF90EF9083
:1026D000DF90CF90BF900C9442104B2D4F70612F24
:1026E000C7010E94AE0226960FB6F894DEBF0FBE59
:1026F000CDBFDF91CF911F910F91FF90EF90DF90B1
:10270000CF90BF900C94F4164B2D4F70612FC701E2
:1027100026960FB6F894DEBF0FBECDBFDF91CF91E6
:102720001F910F91FF90EF90DF90CF90BF900C948E
:10273000E50526960FB6F894DEBF0FBECDBFDF913C
:10274000CF911F910F91FF90EF90DF90CF90BF90AE
:1027500008950E948A190E945F190E94A4190E947C
:10276000B01E0E94001E80E090E00E94740E80E087
:1027700090E00C948A0E0E947A190C94A9130E947E
:10278000AB18292F22952F702C3030F42A3048F4C2
:102790002250223078F405C02C3041F02F3031F037
:1027A00009C0803E48F0803F29F406C093FB88278B
:1027B00080F9089580E0089581E00895CF93DF9334
:1027C00000D000D01F92CDB7DEB70F900F900F90C2
:1027D0000F900F90DF91CF910895CF93DF9300D0AA
:1027E00000D000D0CDB7DEB726960FB6F894DEBF86
:1027F0000FBECDBFDF91CF9108951F93CF93DF938D
:10280000C091790116E080917A01C81799F0D0E063
:102810001C9FF0011D9FF00D1124E558FE4F4081D3
:10282000518162817381848195810E94ED1321968B
:10283000C770E9CFDF91CF911F9108954091AB010F
:102840005091AC016091AD017091AE018091AF01EA
:102850009091B0010C94ED138091B00182958F702E
:1028600009F054C08091AD01882309F44FC08091D4
:102870007901A0917A014091AE015091AF01609130
:10288000AB017091AC01B6E08A1709F43FC090E04B
:1028900041155105C1F17F3F11F46F3FA1F1B89F80
:1028A000F001B99FF00D1124E558FE4F2181271347
:1028B0002AC02081261327C02281211124C0238110
:1028C00034812417350710F421503109241B350BAE
:1028D000283C3105C0F42091B0012F702061209375
:1028E000B00126E0289FF001299FF00D1124E05847
:1028F000FE4F80818F70806180838BEA91E00E941F
:102900009F100C94FD1301968770BECF0895CF924F
:10291000DF92EF92FF920F931F93CF93DF93CDB788
:10292000DEB762970FB6F894DEBF0FBECDBF8C0145
:1029300085E0F801DE011D9601900D928A95E1F780
:10294000D8014C9111965C91119712966C918091DF
:10295000AE019091AF01009709F475C13091AB01C0
:102960007091AC017F3F19F43F3F09F46CC1F8014D
:10297000C380D480E090AD01EE2009F4BEC0209168
:10298000B001C816D90628F0D601A81BB90BCD0195
:1029900004C0809590958C0D9D1DFF24F394883C78
:1029A000910578F0F12C207F09F0C4C07C2DD98AE4
:1029B000C88A89890E94DE138BEA91E00E949F10E9
:1029C000AFC0822F807F09F045C0571313C0431357
:1029D00011C061110FC02F7020612093B0010E94BF
:1029E0001E148BEA91E00E949F108091B001F801C3
:1029F00085832EC0CD2819F15F3F11F44F3FF9F0C8
:102A0000F62E61111CC08091790120917A0136E087
:102A1000821709F45BC090E0389FF001399FF00DF8
:102A20001124E558FE4F7181571306C0708147137A
:102A300003C07281711103C001968770E9CFF62E31
:102A4000662309F41CC18091B00181608093B001BC
:102A5000F12C15C1571309C0431307C0611105C0FC
:102A60008091B001F8018583C8C04D875E878D8550
:102A70009E856A8B0E94BF136A898823D1F16623E1
:102A8000C1F12091B001822F82958F7090E0029762
:102A900074F08091AB019091AC0198878F83198677
:102AA000DB86CA862C87CE0107960E949F1086E09F
:102AB000F801ABEAB1E001900D928A95E1F70E942E
:102AC0002C140E941E14FF24F394D9C04D875E87F6
:102AD0008D859E850E94AB18292F22952F7022305C
:102AE00008F0C1C09F7009F0BBC0805E883008F458
:102AF000C6C0C8010E949F10E6CFC816D90608F4C8
:102B000053C0F601E81BF90BCF01883C910508F48E
:102B100050C0F12C7C2DD98AC88A89890E94DE1385
:102B2000EBEAF1E086E0DF011D928A95E9F70E9469
:102B30001E14A5C0571314C0431312C0611110C056
:102B40008091B001F8018583C8010E949F1086E042
:102B5000EBEAF1E0DF011D928A95E9F7FE2C8FC0C8
:102B60004D875E878D859E856A8B0E94BF136A891B
:102B7000882309F4BECF662309F4BBCF2091B001AE
:102B8000822F82958F7090E002970CF490CF809105
:102B9000AB019091AC019A8389831B82DD82CC8248
:102BA0002E83CE01019681CF809590958C0D9D1D31
:102BB000ACCFF62E662309F49CCF571333C04313D2
:102BC00031C02091B00120FD24C0822F82958F70EA
:102BD000482F50E041155105E1F0D80115962C938E
:102BE00015974F30510549F08F5F982F9295907F40
:102BF000822F8F70892B15968C93C8010E949F108D
:102C000086E0F801ABEAB1E001900D928A95E1F718
:102C10008ECF86E0F801ABEAB1E001900D928A9583
:102C2000E1F72DC04D875E878D859E850E94BF137D
:102C300081113DCF8091B00181608093B001C801C6
:102C40000E949F101CC0662309F453CF4D875E87F6
:102C50008D859E850E94BF13882309F44ACF27CF14
:102C6000811143CF0CC0243008F043CF9F7009F48A
:102C70003CCFD80115969C91907F09F036CF8F2DCF
:102C800062960FB6F894DEBF0FBECDBFDF91CF9135
:102C90001F910F91FF90EF90DF90CF9008951F93B9
:102CA000CF93DF93CDB7DEB72C970FB6F894DEBF86
:102CB0000FBECDBF4F83588769877A878B879C87E4
:102CC000CE0107960E948714882371F08A859B8520
:102CD000892B09F441C088858F3F09F065C08F8139
:102CE0008F3F09F061C038C086E0FE013796DE01F3
:102CF000119601900D928A95E1F76A857B856115A1
:102D0000710551F1FF81E885EF3F11F4FF3F21F19B
:102D100020917A0130E0C90101968770992740918E
:102D2000790150E08417950709F447C0F983EA83D5
:102D30007D836C8396E0929FD001939FB00D112408
:102D4000A558BE4FFE01319601900D929A95E1F77C
:102D500080937A010E94FD1316E080917901909191
:102D60007A018917B9F1189FC001112485589E4F27
:102D70000E948714882371F1E09179011E9FF00170
:102D80001124E558FE4F4081518162817381848115
:102D900095810E94ED138091790190E001968770F2
:102DA000992780937901D9CF4F81588569857A8594
:102DB0008B859C850E94ED13CFCF0E94BB13109290
:102DC0007A0110927901EBEAF1E086E0DF011D92D1
:102DD0008A95E9F72C960FB6F894DEBF0FBECDBFEB
:102DE000DF91CF911F910895EF92FF920F931F9360
:102DF000CF93DF938C01892B09F46CC0F12CEE2466
:102E0000E394E8012196F8018491843740F48430FA
:102E100008F051C0813081F0823019F15BC08537F4
:102E200009F444C0A8F19CE7980F903708F052C00D
:102E30008F770E94421041C00E5F1F4FFE018491A8
:102E400090E2980F983050F48770FE2D01C0FF0F6C
:102E50008A95EAF78F2F0E947D1914C00E947A0F7D
:102E60002DC00E5F1F4FFE01849190E2980F9830A5
:102E700060F48770FE2D01C0FF0F8A95EAF78F2F4F
:102E80000E9483190E94A41919C00E94421016C002
:102E90000E5F1F4FFE01C491CC2381F08FE99FE0AC
:102EA0000197F1F700C00000C150F6CF0E5F1F4F31
:102EB000FE01F49003C00E947A0F8E018F2D8823AB
:102EC00009F49FCFEFE9FFE03197F1F700C0000070
:102ED0008150F5CFDF91CF911F910F91FF90EF902F
:102EE000089508956093B5017093B6018093B7017A
:102EF0009093B8010C94A9130F931F930091B501FF
:102F00001091B6012091B7013091B801DC01CB01DD
:102F1000802B912BA22BB32B8093B5019093B601FC
:102F2000A093B701B093B8011F910F910C94A9130E
:102F30000F931F930091B5011091B6012091B70135
:102F40003091B801DC01CB0180239123A223B3236C
:102F50008093B5019093B601A093B701B093B801E7
:102F60001F910F910C94A9130F931F930091B5011A
:102F70001091B6012091B7013091B801DC01CB016D
:102F800080279127A227B3278093B5019093B6019C
:102F9000A093B701B093B8011F910F910C94A9139E
:102FA0001092B1011092B2011092B3011092B401CB
:102FB0000C94A91341E050E060E070E004C0440FBD
:102FC000551F661F771F8A95D2F74093B101509322
:102FD000B2016093B3017093B4010C94A91341E062
:102FE00050E060E070E004C0440F551F661F771F7B
:102FF0008A95D2F78091B1019091B201A091B3016D
:10300000B091B401482B592B6A2B7B2B4093B10113
:103010005093B2016093B3017093B4010C94A9135F
:1030200041E050E060E070E004C0440F551F661FAF
:10303000771F8A95D2F7409550956095709580914D
:10304000B1019091B201A091B301B091B4014823B4
:1030500059236A237B234093B1015093B2016093BB
:10306000B3017093B4010C94A91341E050E060E007
:1030700070E004C0440F551F661F771F8A95D2F772
:103080008091B1019091B201A091B301B091B401CE
:10309000482759276A277B274093B1015093B201F3
:1030A0006093B3017093B4010C94A9130F931F9311
:1030B0000091B1011091B2012091B3013091B4019E
:1030C000DC01CB01802B912BA22BB32B8093B10180
:1030D0009093B201A093B301B093B4011F910F91EB
:1030E0000C94A9130F931F930091B1011091B20199
:1030F0002091B3013091B401DC01CB0180239123F5
:10310000A223B3238093B1019093B201A093B301A2
:10311000B093B4011F910F910C94A9130F931F93B7
:103120000091B1011091B2012091B3013091B4012D
:10313000DC01CB0180279127A227B3278093B1011F
:103140009093B201A093B301B093B4011F910F917A
:103150000C94A9130895CF92DF92EF92FF920F93F0
:103160001F93CF93DF938C01C090B101D090B20137
:10317000E090B301F090B4018091B5019091B60157
:10318000A091B701B091B801C82AD92AEA2AFB2A2E
:10319000CFE1D0E0D701C6010C2E04C0B695A795AB
:1031A000979587950A94D2F780FF07C0B8018C2FB6
:1031B0000E9409068130910531F4219758F7B80132
:1031C00080E00E940906DF91CF911F910F91FF903F
:1031D000EF90DF90CF90089590910C019923F1F03A
:1031E00090910D019923D1F0982F969596959695EB
:1031F0009F3080F5E0910E01F0910F01E90FF11D74
:10320000877021E030E0A90102C0440F551F8A9564
:10321000E2F7CA019181892B8183089520910E01E3
:1032200030910F01F90132969FEF40E051918517DF
:1032300089F09F3F19F4511101C0942F4F5F4E3018
:10324000A9F79F3F39F0F901E90FF11D97FDFA95B4
:1032500082830895089590910C019923F9F090913B
:103260000D019923D9F0982F9695969596959F30B4
:1032700028F5E0910E01F0910F01E90FF11D877023
:1032800021E030E0A90102C0440F551F8A95E2F702
:10329000CA018095918189238183089520910E012F
:1032A00030910F01F9013296205F3F4F90818913D1
:1032B00001C010823196E217F307C1F7089581E04B
:1032C00090E0E0910E01F0910F01E80FF91F1082DC
:1032D000019680319105A9F708959091CB01892B32
:1032E0008093CB01089580959091CB0189238093A1
:1032F000CB0108951092CB0108959091CA01892BBA
:103300008093CA01089580959091CA018923809382
:10331000CA0108951092CA0108958093B9010895D1
:103320001092B901089580910E0190910F01FC0156
:1033300031969C01205F3F4F80E0919191118F5F0A
:10334000E217F307D1F70895E0910E01F0910F0114
:103350008091CB018083E0910E01F0910F0190816B
:103360008091CA01892B80838091B901882361F003
:10337000E0910E01F0910F019081892B80830E94D2
:10338000931981111092B90180910E0190910F0152
:103390000C945E0ECF92DF92EF92FF926C01EE24BE
:1033A000FF24C114D104E104F10421F0C701B601E6
:1033B00020E101C020E0C72ED82EE92EFF24C11441
:1033C000D104E104F10419F0285FC701B6016B01D3
:1033D0007C0154E0F694E794D794C7945A95D1F7BA
:1033E000C114D104E104F10419F02C5FC701B60146
:1033F0006B017C0142E0F694E794D794C7944A9518
:10340000D1F7C114D104E104F10419F02E5FC70112
:10341000B601DC01CB01B695A79597958795892BC9
:103420008A2B8B2B09F02F5F822FFF90EF90DF907C
:10343000CF9008958091E401843011F120E488E177
:1034400090E00FB6F894A895809360000FBE20938B
:10345000600083B7817F846083BF83B7816083BF4F
:103460007894889583B78E7F83BF0FB6F894A8951C
:1034700080916000886180936000109260000FBEB0
:10348000089508950C94411ACF930E94421A0E9405
:1034900028040E94411AC0E08C2F0E941E05811151
:1034A00004C0CF5FCE30C1F701C081E0CF91089555
:1034B0000E94BB130E94520E0C94480782E084BD08
:1034C00093E095BD9AEF97BD80936E0008952FB756
:1034D000F8948091CD019091CE01A091CF01B0914F
:1034E000D0012FBF0895CF92DF92EF92FF920F93FA
:1034F0001F932FB7F8944091CD015091CE01609168
:10350000CF017091D0012FBF6A017B01EE24FF240F
:103510008C0120E030E0C016D106E206F30610F47C
:10352000415051099A01281B390BC9011F910F9174
:10353000FF90EF90DF90CF9008951F920F920FB6FB
:103540000F9211248F939F93AF93BF938091CD01DE
:103550009091CE01A091CF01B091D0010196A11D13
:10356000B11D8093CD019093CE01A093CF01B09374
:10357000D001BF91AF919F918F910F900FBE0F908F
:103580001F9018950E944A0BF8942FEF87EA91E656
:10359000215080409040E1F700C0000087E090EBB0
:1035A000DC018093ED019093EE01A093EF01B093C5
:1035B000F0019CE088E10FB6F894A8958093600034
:1035C0000FBE90936000FFCFEF92FF920F931F9377
:1035D000CF93DF93D82FC0E08C2F0E941E0500E010
:1035E00010E0E82EF12CC701002E02C095958795BA
:1035F0000A94E2F780FD06C00F5F1F4F06301105E9
:1036000091F709C0602F7C2F80E00E94E6058D13A2
:10361000F3CF81E004C0CF5FCE30F1F680E0DF91E0
:10362000CF911F910F91FF90EF900895CF93C82FE6
:103630008CE20E94E41A882321F08C2FCF910C9405
:10364000E41A80E0CF910895CF930E946B1C811102
:1036500002C00E94511CC5E6C15049F00E942804D6
:103660008FE39CE90197F1F700C00000F5CF89E2F4
:103670000E94161B811113C18AE20E94161B811140
:103680000E94511C85E00E94161B81110E94C21AE3
:103690000E94761C8093CC0187E00E94161B882331
:1036A000A9F18BE10E94161B882351F08091CC0177
:1036B00081FB222720F991E0922790FB81F90EC02F
:1036C0008EE00E94161B882361F08091CC0182FB62
:1036D000222720F991E0922790FB82F98093CC0178
:1036E00015C080E10E94161B9091CC01882341F007
:1036F00093FB222720F981E0822780FB93F904C005
:10370000892F809580FB90F99093CC018091CC011A
:103710000E947A1C0E94881C8093DE0180EE0E9429
:10372000161B882341F08091DE01982F909590FB25
:1037300080F98093DE0189E30E94161B882359F0EB
:103740008091DE0181FB222720F991E0922790FBF6
:1037500081F98093DE0182EE0E94161B882359F0C6
:103760008091DE0182FB222720F991E0922790FBD5
:1037700082F98093DE0186EE0E94161B882359F0A1
:103780008091DE0183FB222720F991E0922790FBB4
:1037900083F98093DE0183EE0E94161B882359F083
:1037A0008091DE0184FB222720F991E0922790FB93
:1037B00084F98093DE0185E30E94161B882359F06B
:1037C0008091DE0185FB222720F991E0922790FB72
:1037D00085F98093DE0181E30E94161B882359F04E
:1037E0008091DE0186FB222720F991E0922790FB51
:1037F00086F98093DE0181E10E94161B882359F02F
:103800008091DE0187FB222720F991E0922790FB2F
:1038100087F98093DE018091DE010E948C1C8091EB
:10382000DE0187FB882780F980930D0187E20E94E3
:10383000161BC82F8EE10E94161B8111C2608FE1FA
:103840000E94161B8111C46080E20E94161B811128
:10385000C86081E20E94161B8111C06182E20E9451
:10386000161B8111C06283E20E94161B8111C06485
:1038700084E20E94161B882311F0C06802C0CC238A
:1038800029F08C2F0E94831C6C2F03C00E947F1C88
:10389000682F70E080E090E0CF910C947217CF9188
:1038A00008956DEE7EEF80E090E00E94C52260E01A
:1038B00082E090E00E94B72260E083E090E00E9406
:1038C000B72260E084E090E00E94B72260E085E0EB
:1038D00090E00C94B72280E090E00E94B12221E0B9
:1038E0008D3E9E4F09F020E0822F089582E090E007
:1038F0000C94A922682F82E090E00C94B72283E018
:1039000090E00C94A922682F83E090E00C94B722F9
:1039100084E090E00C94A922682F84E090E00C945D
:10392000B7228091D30180FF0BC06091130185E025
:10393000689FB001112475956795759567952BC0A3
:1039400081FF09C06091130185E0689FB0011124D7
:103950007595679520C082FF07C06091130185E0CF
:10396000689FB001112417C09091D4019923D1F020
:1039700060911201961788F72091130185E0289F26
:1039800090011124929FA001939F500D112470E08B
:10399000CA010E947B226038710540F461157105EF
:1039A00019F406C065E070E0862F08958FE708954A
:1039B00081E008958091D30180FF08C060911101DA
:1039C00070E0759567957595679521C081FF06C074
:1039D0006091110170E07595679519C082FF04C070
:1039E0006091110170E010C09091D401992399F079
:1039F000609110019617A0F780911101899FC00175
:103A0000112470E00E947B226038710540F461153A
:103A1000710519F406C061E070E0862F08958FE704
:103A2000089581E00895803F21F40E94911C8195C2
:103A300004C0813F29F40E94911C8093D70108950E
:103A4000823F21F40E94911C819504C0833F29F498
:103A50000E94911C8093D6010895893F19F40E9419
:103A6000DA1C05C08A3F31F40E94DA1C81958093EC
:103A7000D80108958B3F21F40E94DA1C819504C07F
:103A80008C3F29F40E94DA1C8093D9010895843F69
:103A900021F48091D501816017C0853F21F4809188
:103AA000D501826011C0863F21F48091D5018460E8
:103AB0000BC0873F21F48091D501886005C0883F05
:103AC00031F48091D50180618093D50108958D3FB7
:103AD00021F48091D30181600BC08E3F21F480914D
:103AE000D301826005C08F3F29F48091D3018460A7
:103AF0008093D3010895803F39F48091D70187FFE7
:103B00006CC01092D70169C0813F29F48091D70120
:103B10001816BCF362C09091D601823F29F497FF3A
:103B20005CC01092D60159C0833F19F41916CCF32A
:103B300054C0893F41F48091D80118160CF04DC053
:103B40001092D8014AC08A3F29F48091D80187FF9A
:103B500044C0F6CF8B3F39F48091D90187FF3DC037
:103B60001092D9013AC08C3F29F48091D9011816DE
:103B7000BCF333C0843F21F48091D5018E7F17C000
:103B8000853F21F48091D5018D7F11C0863F21F4BE
:103B90008091D5018B7F0BC0873F21F48091D501A7
:103BA000877F05C0883F31F48091D5018F7E809357
:103BB000D50113C08D3F21F48091D3018E7F0BC0BE
:103BC0008E3F21F48091D3018D7F05C08F3F29F472
:103BD0008091D3018B7F8093D3018091D601811195
:103BE0000EC08091D70181110AC08091D801811146
:103BF00006C08091D901811102C01092D4010895AC
:103C000085ED91E00E94690E0E94671A9093D2019F
:103C10008093D10108951F93CF93DF938091D101B9
:103C20009091D2010E94731AAC019091D401992312
:103C300021F02091140130E006C0209115018AE0A6
:103C4000289F900111244217530708F485C08091E2
:103C5000D601C091D701D091D8011091D90181111D
:103C600007C0C11175C0D11173C0111171C074C0EA
:103C70009F3F19F09F5F9093D401181624F40E947F
:103C8000911C8093D6018091D60187FF05C00E94C8
:103C9000911C81958093D6011C1624F40E94911CDE
:103CA0008093D7018091D70187FF05C00E94911CA6
:103CB00081958093D7016091D601662331F1C0913F
:103CC000D701CC2311F1062E000C770B880B990B32
:103CD0000E94822123E333E343E35FE30E94E62172
:103CE0000E944A216093D6016C2FCC0F770B880B72
:103CF000990B0E94822123E333E343E35FE30E94B5
:103D0000E6210E944A216093D7011D1624F40E94E7
:103D1000DA1C8093D8018091D80187FF05C00E94EA
:103D2000DA1C81958093D801111624F40E94DA1CC4
:103D30008093D9018091D90187FF05C00E94DA1CC8
:103D400081958093D901DF91CF911F910C94001E32
:103D50009F3F09F08FCFA0CFDF91CF911F910895A2
:103D6000E5EDF1E085E0DF011D928A95E9F710921B
:103D7000D4011092D3010895833081F128F4813069
:103D800059F08230D1F00895853009F449C0B8F176
:103D9000863009F456C0089580911501262F30E031
:103DA000280F311D2F3F310524F4680F6093150152
:103DB00008958FEF80931501089580911401262FA7
:103DC00030E0280F311D2F3F310524F4680F609338
:103DD000140108958FEF80931401089580911301C9
:103DE000262F30E0280F311D2F3F310524F4680FB6
:103DF0006093130108958FEF8093130108958091CC
:103E00001201262F30E0280F311D2F3F310524F4F9
:103E1000680F6093120108958FEF80931201089547
:103E200080911101262F30E0280F311D2F3F3105E1
:103E300024F4680F6093110108958FEF80931101AE
:103E4000089580911001262F30E0280F311D2F3F5B
:103E5000310524F4680F6093100108958FEF80936B
:103E600010010895833011F128F4813049F0823037
:103E700091F00895853081F120F18630C1F10895E7
:103E800080911501681720F4861B80931501089511
:103E900010921501089580911401681720F4861B73
:103EA00080931401089510921401089580911301D4
:103EB000681720F4861B8093130108951092130154
:103EC000089580911201681720F4861B80931201D7
:103ED000089510921201089580911101681720F43D
:103EE000861B80931101089510921101089580910D
:103EF0001001681720F4861B80931001089510921A
:103F0000100108950F931F938D3109F46BC008F0D1
:103F10003FC08E3009F47DC0C0F4873009F46EC014
:103F200068F4863009F0AFC08091CC01817F8E7F2C
:103F30008093CC0181E08093DB01A6C0883009F436
:103F400058C08B3009F49BC09EC0863109F497C0DD
:103F500078F4803109F470C0813109F094C00E9476
:103F6000BB1390910D0181E0892780930D0187C0DB
:103F7000893109F484C08B3109F085C08091CC016E
:103F800081FB222720F991E0922790FB81F94AC01A
:103F9000853309F45BC048F4873209F457C008F44C
:103FA0005AC0893209F452C06EC0833438F48A335F
:103FB00008F067C0883309F462C065C0833409F42F
:103FC00045C0883409F05FC00E94BB130FEF13EDAA
:103FD00020E3015010402040E1F700C000000E94A3
:103FE000C21A4DC00E9404210E94520E0E9448072E
:103FF00046C00E94761C0E94881C41C09091CC0152
:10400000892F817090FF12C0917F9E7F9093CC0189
:104010003BC08091CC0182FB222720F991E09227BE
:1040200090FB82F98093CC01992349F18091CC01D6
:1040300081608093CC0123C08091CC0183FB222737
:1040400020F991E0922790FB83F9ECCF61E070E0DA
:1040500080E090E010C08D5141E050E060E070E001
:104060008A019B0104C0000F111F221F331F8A9574
:10407000D2F7C901B8010E9472170E94BB1381E0F8
:1040800003C08953E9CF80E01F910F91089580E02C
:1040900008950C944720CF93C82F8091DB01813085
:1040A00079F018F08230E9F187C0E0910E01F091CB
:1040B0000F018081813169F0823209F07FC009C02F
:1040C000E0910E01F0910F018081813111F0823277
:1040D00061F48C2F0E944920811104C08C2F0E9412
:1040E000821F1DC081E090E01AC08C2F0E944720E3
:1040F000811114C0C43179F048F4CB3079F0C0316B
:1041000009F060C082E08093DB0108C0C93219F079
:10411000C83321F057C01092DB0154C081E0817098
:1041200053C0C93289F118F5C43171F1A8F4C73010
:1041300009F046C08AE08093150194E19093140140
:1041400093E0909313018093120188E08093110112
:1041500088E28093100134C0CE51C63088F5EC2F30
:10416000F0E0E65DFE4F80818093DA0129C0CE3415
:10417000E9F020F4CB3421F56AE013C0C13579F0C1
:10418000C235F1F461E00DC08091DA01882319F0A5
:104190001092DA0115C081E08093DB0115C061E067
:1041A00006C08091DA010E94BC1E0AC06AE08091BC
:1041B000DA010E94321F04C01092DB0180E004C0CB
:1041C00081E002C080E0ABCFCF910895E1E8F0E05C
:1041D0008081886080838081816080838FB7F8943C
:1041E00093E09093890090ED909388008FBF08959D
:1041F000EFE6F0E08081826080830895EFE6F0E0F2
:1042000080818D7F80830895EFE6F0E0908182E0E9
:104210008927808308951F920F920FB60F92112461
:104220002F933F934F935F936F937F938F939F93BE
:10423000AF93BF93EF93FF938091DC019091DD01E9
:1042400001969093DD018093DC01811103C082E02F
:104250000E944807E091DD01E695E695F0E0E6571B
:10426000FB4FE4918091DC018E1303C080E00E943B
:104270004807FF91EF91BF91AF919F918F917F91EF
:104280006F915F914F913F912F910F900FBE0F90C3
:104290001F9018950E9451216894B1110C94E0214F
:1042A00008950E94C52188F09F5798F0B92F99274B
:1042B000B751B0F0E1F0660F771F881F991F1AF011
:1042C000BA95C9F714C0B13091F00E94DF21B1E076
:1042D00008950C94DF21672F782F8827B85F39F075
:1042E000B93FCCF3869577956795B395D9F73EF4AA
:1042F00090958095709561957F4F8F4F9F4F089552
:10430000E89409C097FB3EF490958095709561956F
:104310007F4F8F4F9F4F9923A9F0F92F96E9BB2725
:104320009395F695879577956795B795F111F8CFA1
:10433000FAF4BB0F11F460FF1BC06F5F7F4F8F4F0C
:104340009F4F16C0882311F096E911C0772321F002
:104350009EE8872F762F05C0662371F096E8862F9A
:1043600070E060E02AF09A95660F771F881FDAF7F1
:10437000880F9695879597F9089557FD9058440FA3
:10438000551F59F05F3F71F04795880F97FB991FB4
:1043900061F09F3F79F08795089512161306140671
:1043A000551FF2CF4695F1DF08C0161617061806FE
:1043B000991FF1CF86957105610508940895E894D9
:1043C000BB2766277727CB0197F908950E94F9212B
:1043D0000C946A220E945C2238F00E94632220F032
:1043E000952311F00C9453220C94592211240C940F
:1043F000E0210E94BD2170F3959FC1F3950F50E01D
:10440000551F629FF001729FBB27F00DB11D639F86
:10441000AA27F00DB11DAA1F649F6627B00DA11D2C
:10442000661F829F2227B00DA11D621F739FB00DD2
:10443000A11D621F839FA00D611D221F749F332742
:10444000A00D611D231F849F600D211D822F762FDB
:104450006A2F11249F5750409AF0F1F088234AF0B8
:10446000EE0FFF1FBB1F661F771F881F9150504024
:10447000A9F79E3F510580F00C9453220C94E02143
:104480005F3FE4F3983ED4F3869577956795B795AB
:10449000F795E7959F5FC1F7FE2B880F911D9695C5
:1044A000879597F9089597F99F6780E870E060E035
:1044B00008959FEF80EC089500240A9416161706BD
:1044C00018060906089500240A9412161306140605
:1044D00005060895092E0394000C11F4882352F068
:1044E000BB0F40F4BF2B11F460FF04C06F5F7F4F20
:1044F0008F4F9F4F089597FB072E16F4009407D017
:1045000077FD09D00E94952207FC05D03EF49095D6
:1045100081959F4F0895709561957F4F0895EE0F97
:10452000FF1F0590F491E02D0994AA1BBB1B51E1DC
:1045300007C0AA1FBB1FA617B70710F0A61BB70B13
:10454000881F991F5A95A9F780959095BC01CD01B8
:104550000895F999FECF92BD81BDF89A992780B54B
:104560000895A8E1B0E042E050E00C94CC22262F60
:10457000F999FECF1FBA92BD81BD20BD0FB6F89448
:10458000FA9AF99A0FBE019608950E94B722272F32
:104590000C94B822DC01CB01FC01F999FECF06C0D6
:1045A000F2BDE1BDF89A319600B40D9241505040F1
:0845B000B8F70895F894FFCF5D
:1045B80020024907D907B40780074C070101BA014F
:1045C80028080A03140A3F4D36394B04FE03C80372
:1045D8008F0322033B0354036D0301020304050602
:0445E80007080900B7
:00000001FF
